:10000000092964001720031801286520A801083079
:10001000A300662017200318A80AAB1EA801A20C93
:10002000A30B0928AB1AA2136620220808003E0879
:1000300084003C0884178004841300052B1B3C06B5
:10004000FF3E0800A400290803190429FF20A0008E
:100050002518831724088400200880008313A40A2D
:10006000A9032328A6003E0884008030BB05083081
:10007000A70003100318BB0A4B20A60CA70B3A28B5
:100080000000AB1A3B0C4B20072103144B202F0818
:10009000A3002E0876288413AB1F5A2800083C04BE
:1000A0002B1F3C068000841700083C04031C3C0600
:1000B0008000662800083C04031C3C062B1B3C0601
:1000C000800084173C09800566283B172B081F39E0
:1000D000003EA1002A08083E0318A10A3B1F8328FE
:1000E0003B13A00002309A208328A301A200FF3016
:1000F000A207031CA307031C04290330A100E4305A
:1001000083207728A101F63EA000A109031C8E28B8
:10011000FE300000A00703188928A0076400A10F83
:10012000882800002018942820189628080003101A
:10013000A10CA00CFF3E0318972820080429A10158
:10014000A301A2000230B228A2000330B228A2000C
:100150000130B228A2000630B228A2000430B22832
:10016000A2000530A80023082102031DB928220897
:100170002002043003180130031902302805031D42
:10018000FF3004290038031DFF300405031DFF3034
:1001900004290404031DFF300429A501A401103023
:1001A000A600210DA40DA50D2208A4022308031CFE
:1001B000230FA5020318E3282208A4072308031825
:1001C000230FA5070310A00DA10DA60BD128200811
:1001D00004291030A800A101A001A70CA60C031C43
:1001E000F7282208A00723080318230FA107A10C52
:1001F000A00CA50CA40CA80BED282408042984004D
:1002000031088A00300882008313031383126400CC
:10021000080083163F308500403086008701063095
:100220009F008030810083128B010430920083167E
:10023000FF309200831295019B010C3097000C3027
:100240009D008316AC0183120612831606128312D8
:1002500087138316871383120130A3002C308A0181
:100260007620871783168713643083128A017520DE
:1002700086158316861183120614831606108312C0
:100280000616831606128312861483168610FA3019
:10029000A800A90128088312950064308A017520FE
:1002A0008A110A12112364308A0175200630BE00BB
:1002B0004030BC002030AA00AB011530A90001304D
:1002C000B000B101A50155308A0122208316AA0190
:1002D00083126400163083162A028A110A128312CE
:1002E00003188E2983162A08553E840000088312BD
:1002F000B200D0303207B200FF300318013EB30025
:1003000083162A08403E8400831232088000831638
:10031000AA0A8A110A128312031D69294108A6003C
:10032000A7010A30A200A3018A01E920B200250832
:10033000B3004208B2070318B30A4008A600A70199
:100340006430A200A3018A01E920B4002508B500A9
:100350003208B40733080318013EB5073408A60075
:100360003508A7001930A200A3018A01E920B400D2
:100370002508B5003408A0003508A1000A30A20005
:10038000A3018A01CD208316A600831221088316BB
:10039000A70083124408A600A7010A30A200A30107
:1003A0008A01E920B2002508B3004508B207031806
:1003B000B30A4308A600A7016430A200A3018A0182
:1003C000E920B4002508B5003208B4073308031843
:1003D000013EB5073408A6003508A7001930A20071
:1003E000A3018A01E920B4002508B5003408A00063
:1003F0003508A1000A30A200A3018A01CD2083168E
:10040000A800831221088316A90083125408A600AD
:10041000A7012830A200A3018A01E920B200250823
:10042000B300203032078316A20003300318013EC8
:10043000831233078316A30083124808A600A7017E
:100440000A30A200A3018A01E920B2002508B30006
:100450004908B2070318B30A4708A600A701643089
:10046000A200A3018A01E920B4002508B5003208E2
:10047000B40733080318013EB5074608A600A701D4
:10048000E830A2000330A3008A01E920B600250865
:10049000B70034083607EA0035080318013E37076D
:1004A000EB00640083162C08013C8A110A128312A7
:1004B000031D5E2A8316260883129B0083162808D4
:1004C000831295006A08A0006B08A100A301003008
:1004D0008A01B0208A110A12031D712A8A110A1298
:1004E00011236A08A0006B08A100A30165308A01EE
:1004F000B0208A110A12031D802A8A110A1256247A
:100500006A08A0006B08A100A301CA308A01B020CC
:100510008A110A12031D8F2A8A110A12D4236A082B
:10052000A0006B08A1000130A3002F308A01B02089
:100530008A110A12031D9F2A8A110A12F9236A08D6
:10054000A0006B08A1000130A30094308A01B02004
:100550008A110A12031DAF2A8A110A122C246A0872
:10056000A0006B08A1000130A300F9308A01B0207F
:100570008A110A12031DBF2A8A110A1242246A082C
:10058000A0006B08A1000230A3005E308A01B020F9
:100590008A110A12031DCF2A8A110A122C276A080F
:1005A000A0006B08A1000230A300C3308A01B02074
:1005B0008A110A12031DDF2A8A150A126A216A08A3
:1005C000A0006B08A1000330A30028308A01B020EE
:1005D0008A110A12031DEF2A8A150A120D226A08CF
:1005E000A0006B08A1000330A3008D308A01B02069
:1005F0008A110A12031DFF2A8A150A12A9226A0803
:10060000A0006B08A1000430A30057308A01B0207D
:100610008A110A12031D0F2B8A150A1261238A01FF
:10062000562907128316071283128716831687121C
:1006300064008A110A128312051A202B8A01112BD9
:1006400087128316871283128615831686118312EA
:10065000061483160610AA018312640065308316FF
:100660002A028A110A12831203185B2B8612831640
:10067000861283120611831606118312071383163E
:100680000713323083128A0182208616831686125F
:100690008312061583160611831207178316071394
:1006A000FA3083128A0182208316AA0A8A110A125A
:1006B0008312031D2D2B0130A3002C308A017620DC
:1006C0008611831686118312061083160610831274
:1006D000861283168612323083128A018220861691
:1006E00083168612FA3083128A01822064008A11EE
:1006F0000A1285197D2B8A01682BFA01FB0164001F
:100700008A110A128518882B061183160611831286
:1007100064008A110A120519912B07138316071317
:10072000831232308A018220061583160611831245
:10073000071783160713FA3083128A0182200030CC
:1007400085180130A00000308A019F20B2000030DF
:1007500005190130A00000308A019F20B400320842
:10076000840034088A01C920B400B500640034084C
:1007700035048A110A120319BF2B8A017F2BFC0151
:10078000FD01C8308A0175200630BE008030BC00F3
:100790001E30AA00AB01AE01AF014F308A013220FA
:1007A0004B308A0132200800FF3095000712831673
:1007B0000712831287168316871264008A110A12A1
:1007C0008312051AE52B8A01D42B87128316871210
:1007D00006308312BE008030BC001E30AA00AB0180
:1007E000AE01AF014F308A0132204B308A013220F6
:1007F00008008316280883129500640083162C08CD
:10080000013C8A110A128312031D1C2C87128316C5
:100810008712831207168316071264008A110A12C0
:100820008312851A152C8A01F92B071283160712D9
:10083000C83083128A0175200630BE008030BC00AB
:100840001E30AA00AB01AE01AF014F308A01322049
:100850004B308A013220080083160130AC00260894
:1008600083129B000630BE008030BC001E30AA0000
:10087000AB01AE01AF014F308A0132204B308A010B
:10088000322008008316AC0183129B010630BE00A3
:100890008030BC001E30AA00AB01AE01AF014F306A
:1008A0008A0132204B308A01322008008316013041
:1008B000AC00260883129B004D08A600A7010A3051
:1008C000A200A3018A01E920B2002508B3004E0866
:1008D000B2070318B30A4C08A600A7016430A200AF
:1008E000A3018A01E920B4002508B5003208B40745
:1008F00033080318013EB5074B08A600A701E830EE
:10090000A2000330A3008A01E920B6002508B70041
:100910003408B60735080318013EB7074A08A60091
:10092000A7011030A2002730A3008A01E920B800F7
:100930002508B90036083807FE0037080318013EBD
:100940003907FF005208A600A7010A30A200A30140
:100950008A01E920B2002508B3005308B207031842
:10096000B30A5108A600A7016430A200A3018A01BE
:10097000E920B4002508B5003208B407330803188D
:10098000013EB5075008A600A701E830A2000330D9
:10099000A3008A01E920B6002508B7003408B6078D
:1009A00035080318013EB7074F08A600A70110300D
:1009B000A2002730A3008A01E920B8002508B90069
:1009C000360838078316A000831237080318013E43
:1009D00039078316A10083127E08A0007F08A100BA
:1009E0007B08A3007A088A01A120B20083162008A0
:1009F0008312A000831621088312A1007D08A300A2
:100A00007C088A01A120B4003208840034088A01DD
:100A1000C220B400B5006400340835048A110A12FB
:100A20000319182D83162B1483128A110A121B2DF9
:100A300083162B1083127E08A0007F08A1007B087C
:100A4000A3007A088A01AA208A110A12031D342DF4
:100A50007A087E02F4007B08031C013E7F02F50049
:100A600086158316861183127E08A0007F08A100D8
:100A70007B08A3007A088A01A4208A110A12031DA8
:100A80004D2D7E087A02F4007F08031C013E7B0294
:100A9000F50086118316861183127E08A0007F0858
:100AA000A1007B08A3007A088A01B0208A110A12EB
:100AB000031D5C2DF401F501831620088312A000AC
:100AC000831621088312A1007D08A3007C088A01F7
:100AD000AA208A110A12031D7D2D7C08831620028C
:100AE0008312F6007D08031C013E83162102831247
:100AF000F70006148316061083128316200883124B
:100B0000A000831621088312A1007D08A3007C08A1
:100B10008A01A4208A110A12031D9E2D8316200823
:100B200083127C02F60083162108031C013E831207
:100B30007D02F70006108316061083128316200824
:100B40008312A000831621088312A1007D08A30050
:100B50007C088A01B0208A110A12031DB12DF6010A
:100B6000F70183162208A4002308A5008312740845
:100B7000F0007508F1007608F2007708F3007408B9
:100B8000A0007508A100A30100308A01AA208A11E3
:100B90000A12031DD52D8612831686120130831288
:100BA000F4020030031C013EF5027608A00077082D
:100BB000A100A30100308A01AA208A110A12031D94
:100BC000EF2D0611831606118312071383160713E0
:100BD00001308312F6020030031C013EF70214308C
:100BE0008A018220861683168612831206158316C2
:100BF0000611831207178316071383127008A000CB
:100C00007108A1000130A30040308A01AD20B2007C
:100C10007208A0007308A1000130A30040308A01CF
:100C2000AD20B4003208840034088A01C920B40021
:100C3000B5006400340835048A110A120319302EF5
:100C4000643083162402A2000030031C013E2502FA
:100C5000A30083128A110A12932E8A110A12932E6C
:100C60007408A0007508A100A30196308A01AD2088
:100C7000B2007608A0007708A100A30196308A018F
:100C8000AD20B4003208840034088A01C920B400C1
:100C9000B5006400340835048A110A1203196E2E57
:100CA000831622088312A000831623088312A10052
:100CB000831625088312A3008316240883128A0151
:100CC000A4208A110A12031D6B2E0A308316A20774
:100CD0000318A30A83128A110A12932E2030831656
:100CE00024028312B2000330031C013E8316250246
:100CF0008312B300831622088312A00083162308F0
:100D00008312A1003308A30032088A01AA208A11A5
:100D10000A12031D932E06308316A2020030031C14
:100D2000013EA3028312831623088312A1008316B7
:100D3000220883128A0183207408A0007508A1008C
:100D4000A30100308A01A120B2007608A000770834
:100D5000A100A30100308A01A120B4003208840060
:100D600034088A01C220B400B50064003408350498
:100D70008A110A120319CB2E7E08FA007F08FB00A5
:100D8000831620088312FC00831621088312FD00BD
:100D90008A110A12CD2E8A01BF2D83162C088312C8
:100DA000A00001308A019F20B200831600302B186A
:100DB00001308312A00000308A019F20B400320865
:100DC000840034088A01C220B400B50064003408ED
:100DD00035048A110A1203191C2F8316280883125E
:100DE000950087128316871283120716831607123F
:100DF00064008A110A128312851A002F8A01CD2EEF
:100E00000712831607128312FF3095008716831688
:100E10008712831207128316071264008A110A12BE
:100E20008312051A152F8A01042F87128316871241
:100E300083128A110A121C2F0630BE008030BC00BB
:100E40001E30AA00AB01AE01AF014F308A01322043
:100E50004B308A01322008008316AC0183129B01BB
:100E600007128316071283128716831687126400EF
:100E70008A110A128312051A3F2F8A012C2F87121A
:100E80008316871283128615831686118312061421
:100E900083160610AA0183126400653083162A02A5
:100EA0008A110A12831203187A2F86128316861269
:100EB0008312061183160611831207138316071374
:100EC000323083128A01822086168316861283129C
:100ED0000615831606118312071783160713FA30B7
:100EE00083128A0182208316AA0A8A110A128312A7
:100EF000031D4C2F0130A3002C308A01762086116F
:100F0000831686118312061083160610831286122A
:100F100083168612323083128A0182208616831647
:100F20008612FA3083128A01822064008A110A1222
:100F300085199C2F8A01872FFA01FB0164008A1111
:100F40000A128518A72F0611831606118312640052
:100F50008A110A120519B02F07138316071383127B
:100F600032308A0182200615831606118312071774
:100F700083160713FA3083128A0182200030851805
:100F80000130A00000308A019F20B2000030051916
:100F90000130A00000308A019F20B4003208840094
:100FA00034088A01C920B400B5006400340835044F
:100FB0008A110A120319DE2F8A019E2FFC01FD01FE
:100FC0000130A3002C308A0176204D08A600A7012D
:100FD0000A30A200A3018A01E920B2002508B3006B
:100FE0004E08B2070318B30A4C08A600A7016430E4
:100FF000A200A3018A01E920B4002508B500320847
:10100000B40733080318013EB5074B08A600A70133
:10101000E830A2000330A3008A01E920B6002508C9
:10102000B7003408B60735080318013EB7074A0869
:10103000A600A7011030A2002730A3008A01E920F2
:10104000B8002508B90036083807FE00370803182D
:10105000013E3907FF005208A600A7010A30A2008E
:10106000A3018A01E920B2002508B3005308B207A2
:101070000318B30A5108A600A7016430A200A30117
:101080008A01E920B4002508B5003208B407330806
:101090000318013EB5075008A600A701E830A200DA
:1010A0000330A3008A01E920B6002508B700340800
:1010B000B60735080318013EB7074F08A600A70179
:1010C0001030A2002730A3008A01E920B8002508CB
:1010D000B900360838078316A000831237080318B2
:1010E000013E39078316A10083127E08A0007F0805
:1010F000A1007B08A3007A088A01AA208A150A1297
:10110000031D8E287A087E02F4007B08031C013E32
:101110007F02F50086158316861183127E08A000D3
:101120007F08A1007B08A3007A088A01A4208A1501
:101130000A12031DA7287E087A02F4007F08031C08
:10114000013E7B02F50086118316861183128316F9
:1011500020088312A000831621088312A1007D08B5
:10116000A3007C088A01AA208A150A12031DC82838
:101170007C08831620028312F6007D08031C013EC2
:10118000831621028312F7000614831606108312B9
:10119000831620088312A000831621088312A10061
:1011A0007D08A3007C088A01A4208A150A12031D69
:1011B000E9288316200883127C02F6008316210892
:1011C000031C013E83127D02F700061083160610F1
:1011D00083127408A0007508A100A30100308A01E1
:1011E000AA208A150A12031DFF288612831686126A
:1011F00001308312F4020030031C013EF502760830
:10120000A0007708A100A30100308A01AA208A1556
:101210000A12031D192906118316061183120713DA
:101220008316071301308312F6020030031C013EBF
:10123000F70232308A0182208616831686128312C4
:101240000615831606118312071783160713FA3043
:1012500083128A0182207408A0007508A100A301EE
:1012600000308A01A720B2007608A0007708A1000C
:10127000A30100308A01A720B4003208840034089A
:101280008A01C920B400B5006400340835048A1509
:101290000A1203195A297E08FA007F08FB008316F8
:1012A00020088312FC00831621088312FD008A1592
:1012B0000A12E9280630BE008030BC001E30AA00A9
:1012C000AB01AE01AF014F308A0132204B308A01B1
:1012D000322008004D08A600A7010A30A200A30191
:1012E0008A01E920B2002508B3004E08B2070318AE
:1012F000B30A4C08A600A7016430A200A3018A012A
:10130000E920B4002508B5003208B40733080318F3
:10131000013EB5074B08A600A701E830A200033044
:10132000A3008A01E920B6002508B7003408B607F3
:1013300035080318013EB7074A08A600A701103078
:10134000A2002730A3008A01E920B8002508B900CF
:1013500036083807FE0037080318013E3907FF003A
:10136000FF30950007128316071283128716831623
:10137000871264008A150A128312051AC2298A1577
:101380000A126A298712831687128312F801F9015B
:101390008611831686118312F80A0319F90A64006C
:1013A0008A150A128519D829861283168612831285
:1013B000F430831622028312B2000130031C013E76
:1013C000831623028312B3003308A10032088A0176
:1013D000832086168316861283127808A000790867
:1013E000A1007F08A3007E088A01A4208A150A12A2
:1013F000031DFD298A150A12C8290630BE00803057
:10140000BC001E30AA00AB01AE01AF014F308A0113
:1014100032204B308A01322008004D08A600A70177
:101420000A30A200A3018A01E920B2002508B30016
:101430004E08B2070318B30A4C08A600A70164308F
:10144000A200A3018A01E920B4002508B5003208F2
:10145000B40733080318013EB5074B08A600A701DF
:10146000E830A2000330A3008A01E920B600250875
:10147000B7003408B60735080318013EB7074A0815
:10148000A600A7011030A2002730A3008A01E9209E
:10149000B8002508B90036083807FE0037080318D9
:1014A000013E3907FF00FF3095000712831607122F
:1014B000831287168316871264008A150A12831214
:1014C000051A652A8A150A120D2A871283168712B1
:1014D0008312F801F9018615831686118312F80A22
:1014E0000319F90A861283168612F4302202831237
:1014F000B2000130031C013E831623028312B300A5
:101500003308A10032088A018320861683168612CA
:1015100083127808A0007908A1007F08A3007E0844
:101520008A01A4208A150A12031D992A8A150A1213
:101530006B2A0630BE008030BC001E30AA00AB0112
:10154000AE01AF014F308A0132204B308A01322088
:1015500008005208A600A7010A30A200A3018A01D0
:10156000E920B2002508B3005308B2070318B30AF4
:101570005108A600A7016430A200A3018A01E92056
:10158000B4002508B5003208B40733080318013E3B
:10159000B5075008A600A701E830A2000330A30059
:1015A0008A01E920B6002508B7003408B6073508D7
:1015B0000318013EB7074F08A600A7011030A2008C
:1015C0002730A3008A01E920B8002508B9003608B1
:1015D00038078316A000831237080318013E390725
:1015E0008316A1008312FF3095000712831607129D
:1015F000831287168316871264008A150A128312D3
:10160000051A052B8A150A12A92A87128316871232
:101610008312F801F9010610831606108312F80AE6
:101620000319F90A64008A150A1285181B2B061182
:1016300083160611831264008A150A120519242BD9
:101640000713831607138312F430831622028312C2
:10165000B2000130031C013E831623028312B30043
:101660003308A10032088A0183200615831606116B
:10167000831207178316071383127808A0007908CE
:10168000A100831621088312A30083162008831269
:101690008A01A4208A150A12031D512B8A150A12E9
:1016A0000B2B0630BE008030BC001E30AA00AB0100
:1016B000AE01AF014F308A0132204B308A01322017
:1016C00008005208A600A7010A30A200A3018A015F
:1016D000E920B2002508B3005308B2070318B30A83
:1016E0005108A600A7016430A200A3018A01E920E5
:1016F000B4002508B5003208B40733080318013ECA
:10170000B5075008A600A701E830A2000330A300E7
:101710008A01E920B6002508B7003408B607350865
:101720000318013EB7074F08A600A7011030A2001A
:101730002730A3008A01E920B8002508B90036083F
:1017400038078316A000831237080318013E3907B3
:101750008316A1008312FF3095000712831607122B
:10176000831287168316871264008A150A12831261
:10177000051ABD2B8A150A12612B87128316871250
:101780008312F801F9010614831606108312F80A71
:101790000319F90A0611831606118312071383161B
:1017A0000713F43022028312B2000130031C013E01
:1017B000831623028312B3003308A10032088A0182
:1017C0008320061583160611831207178316071345
:1017D00083127808A0007908A100831621088312DB
:1017E000A3008316200883128A01A4208A150A12F6
:1017F000031DFD2B8A150A12C32B0630BE00803054
:10180000BC001E30AA00AB01AE01AF014F308A010F
:1018100032204B308A013220080063008A150A12F8
:021820000D2C8D
:02400E007D3FF4
:00000001FF
